:100000000C9462000C948A000C948A000C948A0070
:100010000C948A000C948A000C948A000C948A0038
:100020000C948A000C948A000C948A000C948A0028
:100030000C948A000C948A000C948A000C948A0018
:100040000C9487040C948A000C9429060C948A0062
:100050000C948A000C948A000C948A000C948A00F8
:100060000C948A000C948A000000000024002700F1
:100070002A0000000000250028002B0000000000DE
:1000800023002600290004040404040404040202DA
:100090000202020203030303030301020408102007
:1000A0004080010204081020010204081020000012
:1000B0000007000201000003040600000000000029
:1000C0000000AE0711241FBECFEFD4E0DEBFCDBFCE
:1000D00011E0A0E0B1E0ECEBF3E102C005900D927D
:1000E000AE33B107D9F712E0AEE3B1E001C01D9223
:1000F000AA31B107E1F710E0C4ECD0E004C02297C8
:10010000FE010E94D809C23CD107C9F70E948004B1
:100110000C94DC090C940000FB01DC0104C08D91FF
:100120000190801921F441505040C8F7881B990B69
:100130000895EF92FF920F931F93CF93DF938091D7
:100140003E0190913F01181619061CF0C0E0D0E066
:1001500045C0EE24FF2487012CC08091000161E09E
:100160000E948D0580913E0190913F0162E070E018
:100170000E947209CB010E9407058091000160E096
:100180000E948D0580913E0190913F0162E070E0F8
:100190000E947209CB010E94070580913E01909157
:1001A0003F01AA2797FDA095BA2FE80EF91E0A1F56
:1001B0001B1F8091420190914301A0914401B09195
:1001C0004501E816F9060A071B073CF20EC08091AC
:1001D0004201909143010E940705219680912401DC
:1001E00090912501C817D90794F3DF91CF911F9102
:1001F0000F91FF90EF900895EF92FF920F931F934E
:10020000CF93DF9386E1E82E81E0F82E08E111E03C
:10021000C0E0D0E02FC0F701819191917F019093D0
:100220003F0180933E01F801619171918F017093BC
:10023000410160934001882777FD8095982F209198
:100240001E0130911F0140912001509121010E9417
:10025000530960934201709343018093440190934A
:1002600045010E94990080912201909123010E94F2
:100270000705219680911C0190911D01C817D9078F
:1002800054F2DF91CF911F910F91FF90EF9008955D
:10029000EF92FF920F931F93CF93DF9322E0E22E12
:1002A00021E0F22E0CE011E0C0E0D0E02FC0F70119
:1002B000819191917F0190933F0180933E01F801DC
:1002C000619171918F017093410160934001882782
:1002D00077FD8095982F20911E0130911F0140914C
:1002E0002001509121010E945309609342017093B3
:1002F000430180934401909345010E9499008091AD
:100300002201909123010E940705219680911A01F4
:1003100090911B01C817D90754F2DF91CF911F911B
:100320000F91FF90EF900895EF92FF921F93CF935C
:10033000DF93182F7B0161E00E946D05C0E0D0E0E3
:1003400015C0812F61E00E948D0568EC70E080E0AF
:1003500090E00E94DD04812F60E00E948D0568EC32
:1003600070E080E090E00E94DD042196CE15DF056C
:1003700044F3DF91CF911F91FF90EF9008950E9479
:10038000CF049B01AC0120936A0130936B01409331
:100390006C0150936D0180916E0190916F01A0915D
:1003A0007001B0917101281B390B4A0B5B0B57FF91
:1003B00007C050954095309521953F4F4F4F5F4F67
:1003C000209372013093730140937401509375012F
:1003D0008091260190912701A0912801B0912901D7
:1003E00082179307A407B50724F580912C010E947A
:1003F0004F0590935F0180935E018756924024F4ED
:1004000080912A0160E003C080912A0161E00E948E
:100410008D0580916A0190916B01A0916C01B09162
:100420006D0180936E0190936F01A0937001B09362
:1004300071010895109269011092680145C087E02A
:1004400092E00E94730780935E0190935F01209178
:10045000680130916901F901EA5BFE4F80832F5FEB
:100460003F4F30936901209368012A30310561F5CF
:1004700086E491E060E571E04AE050E00E948C0083
:10048000009719F40E94FC001FC020E030E0F90141
:10049000E05BFE4FD901AA5BBE4F8C9180832F5F3A
:1004A0003F4F2A30310599F780914D0180935A01D1
:1004B00080914E0180935B0180914F0180935C019C
:1004C00010925D010E94480187E092E00E945F0760
:1004D000882309F0B4CF0895AF92BF92CF92DF92F4
:1004E000EF92FF920F931F93E62EC82EDD2454E067
:1004F000CC0CDD1C5A95E1F7FF2447E0A42E42E026
:10050000B42EA70134E0559547953A95E1F74C296B
:100510005D29662757FD6095762FC50120E030E004
:100520000E94F5086091300170913101882777FDB4
:100530008095982F0E94DD048FE0E822FF24EC28AC
:10054000FD280027F7FC0095102FC501B801A70171
:1005500020E030E00E94F508609130017091310197
:10056000882777FD8095982F0E94DD041F910F91B9
:10057000FF90EF90DF90CF90BF90AF9008952F92B3
:100580003F925F926F927F928F929F92AF92BF92B3
:10059000CF92DF92EF92FF920F931F93A7E02A2E44
:1005A000A2E03A2E4091780150917901406F662780
:1005B00057FD6095762FC10120E030E00E94F508DC
:1005C0008091780160915A010E946C0280917801BB
:1005D00060915B010E946C028091780160915C01E6
:1005E0000E946C025090780100D000D060916001B0
:1005F00070916101882777FD8095982FFFEF6F2E0E
:10060000712C812C912CEDB7FEB7618272828382AE
:10061000948220E030E040E050E0E3EAEE2EE2E0B9
:10062000FE2E012D112DAA24BB2465010E940A096A
:100630000F900F900F900F90852D0E946C0250909C
:10064000780100D000D06091620170916301882729
:1006500077FD8095982FEDB7FEB761827282838215
:10066000948220E030E040E050E00E940A090F90C0
:100670000F900F900F90852D0E946C025090780182
:1006800000D000D06091640170916501882777FDEA
:100690008095982FEDB7FEB7618272828382948233
:1006A00020E030E040E050E00E940A090F900F90F7
:1006B0000F900F90852D0E946C025090780100D011
:1006C00000D06091660170916701882777FD809561
:1006D000982FEDB7FEB7618272828382948220E008
:1006E00030E040E050E00E940A090F900F900F9018
:1006F0000F90852D0E946C02C1010E941F0860911D
:10070000300170913101882777FD8095982F0E94E4
:10071000DD041F910F91FF90EF90DF90CF90BF907D
:10072000AF909F908F907F906F905F903F902F90B1
:10073000089580E00E944F059093610180936001CD
:1007400081E00E944F05909363018093620182E0F3
:100750000E944F05909365018093640184E00E949C
:100760004F0590936701809366010E94BF02089530
:100770000E941A020E9499030E94BF0162E370E086
:1007800080E090E00E94DD040895EF92FF920F93C5
:100790001F93CF93DF9387E092E040E855E260E05B
:1007A00070E00E9466068091000161E00E946D0584
:1007B00080912A0161E00E946D0580912E0161E027
:1007C0000E946D0580912E0161E00E948D0585E0FB
:1007D00090E008C060E00E946D05809176019091E4
:1007E000770101969093770180937601809176014D
:1007F00090917701893091056CF385E090E09093BA
:10080000770180937601B4E0EB2EF12C02E010E04A
:10081000C1E0D0E03EC00E94DA05892B89F18091C9
:100820007601909177018530910529F4D0935F018D
:10083000C0935E0117C08630910529F410935F01C3
:1008400000935E010FC08730910529F4F0925F019B
:10085000E0925E0107C08830910521F490935F011A
:1008600080935E01809178019091790120915E01E1
:1008700030915F01820F931F9093790180937801EB
:100880008091760190917701019690937701809302
:1008900076018091760190917701893091050CF471
:1008A000BACF84E090E090937901809378018DE055
:1008B00090E063E070E00E9494010E944801109271
:1008C0005A0110925B0110925C0110925D0180E070
:1008D00090E0FC01EA5BFE4F1082FC01E05BFE4F02
:1008E0001082019689309105A1F710924F01109264
:1008F0005901DF91CF911F910F91FF90EF900895D3
:100900000E9415050E94C5030E94B803FDCF1F92E7
:100910000F920FB60F9211242F933F938F939F93B3
:10092000AF93BF9380917E0190917F01A091800150
:10093000B0918101309182010196A11DB11D232F3B
:100940002D5F2D3720F02D570196A11DB11D20934D
:10095000820180937E0190937F01A0938001B093E8
:10096000810180917A0190917B01A0917C01B091ED
:100970007D010196A11DB11D80937A0190937B01A9
:10098000A0937C01B0937D01BF91AF919F918F9116
:100990003F912F910F900FBE0F901F9018958FB71A
:1009A000F89420917E0130917F0140918001509117
:1009B00081018FBFB901CA010895EF92FF920F9391
:1009C0001F937B018C018FB7F89440917E01509169
:1009D0007F0160918001709181018FBF2FB7F894E2
:1009E00080917E0190917F01A0918001B091810161
:1009F0002FBF841B950BA60BB70BE816F9060A0749
:100A00001B0760F71F910F91FF90EF9008950197DA
:100A100059F0FC01EE0FFF1FEE0FFF1F32978FB74B
:100A2000F8943197F1F78FBF0895789484B5826078
:100A300084BD84B5816084BD85B5826085BD85B582
:100A4000816085BDEEE6F0E0808181608083E1E831
:100A5000F0E0808182608083808181608083E0E833
:100A6000F0E0808181608083E1EBF0E08081846050
:100A70008083E0EBF0E0808181608083EAE7F0E052
:100A800080818460808380818260808380818160B6
:100A900080838081806880831092C10008958F7068
:100AA000909132019295990F990F907C982B909389
:100AB0007C0080917A00806480937A0080917A0033
:100AC00086FDFCCF2091780040917900942F80E042
:100AD00030E0282B392BC9010895282F30E0C901B7
:100AE00086569F4FFC0194912A573F4FF9018491FC
:100AF000882391F0E82FF0E0EE0FFF1FE859FF4F39
:100B0000A591B491662329F48C91909589238C93B7
:100B100008958C91892B8C930895482F50E0CA0139
:100B200082559F4FFC012491CA0186569F4FFC01BC
:100B300094914A575F4FFA0134913323D1F1222324
:100B400031F1233021F4809180008F7705C024306B
:100B500031F4809180008F7D8093800018C0213017
:100B600019F484B58F7704C0223021F484B58F7DC9
:100B700084BD0DC0263021F48091B0008F7705C070
:100B8000273029F48091B0008F7D8093B000E32F4F
:100B9000F0E0EE0FFF1FEE58FF4FA591B4916623D2
:100BA00029F48C91909589238C9308958C91892BAD
:100BB0008C930895682F70E0CB0182559F4FFC0104
:100BC0002491CB0186569F4FFC0144916A577F4F79
:100BD000FB019491992319F420E030E038C02223DE
:100BE00031F1233021F4809180008F7705C02430CB
:100BF00031F4809180008F7D8093800018C0213077
:100C000019F484B58F7704C0223021F484B58F7D28
:100C100084BD0DC0263021F48091B0008F7705C0CF
:100C2000273029F48091B0008F7D8093B000892F08
:100C300090E0880F991F84589F4FFC01A591B491B3
:100C40008C9120E030E0842311F021E030E0C901F4
:100C500008951F920F920FB60F9211242F933F9376
:100C60004F935F936F937F938F939F93AF93BF93B4
:100C7000EF93FF934091C600E0910302F0910402CC
:100C8000CF01019660E870E00E9472099C0180919A
:100C90000502909106022817390739F0ED57FE4FEB
:100CA00040833093040220930302FF91EF91BF91A0
:100CB000AF919F918F917F916F915F914F913F91F4
:100CC0002F910F900FBE0F901F9018955F926F920B
:100CD0007F928F929F92AF92BF92CF92DF92EF92CC
:100CE000FF920F931F93CF93DF93EC013A014B01D7
:100CF000413482E458078FE0680780E078070CF001
:100D00007FC060E874E88EE190E0A40193010E9446
:100D1000A7092150304040405040CA01B90122E0AB
:100D200030E040E050E00E94A70959016A01A601A5
:100D30009501209530954095509594E0220F331FF2
:100D4000441F551F9A95D1F760E074E284EF90E05C
:100D50000E94A709CA01B9012FEF30E040E050E03E
:100D60000E945309A40193010E94A709C90181505F
:100D70009F4F181619061CF4522E5A9403C055247E
:100D80005394521A60E079E08DE390E0A40193015E
:100D90000E94A7092150304040405040CA01B9018B
:100DA00022E030E040E050E00E94A7092095309515
:100DB0004095509583E0220F331F441F551F8A959D
:100DC000D1F760E074E284EF90E00E94A709CA01C5
:100DD000B9012FEF30E040E050E00E945309A40138
:100DE00093010E94A709C90181509F4F1816190647
:100DF0001CF4822F815002C081E0821B851500F512
:100E0000E885F98581E090E00A8802C0880F991F83
:100E10000A94E2F7808360E079E08DE390E0A4013A
:100E200093010E94A7092150304040405040CA0120
:100E3000B90122E030E040E050E00E94A70904C080
:100E4000E885F98510829501EC81FD813083EE8182
:100E5000FF812083EA85FB85208141E050E0CA01C3
:100E60000E8402C0880F991F0A94E2F7282B208372
:100E7000EA85FB852081CA010F8402C0880F991F73
:100E80000A94E2F7282B2083EA85FB858081088875
:100E900002C0440F551F0A94E2F7842B8083DF9130
:100EA000CF911F910F91FF90EF90DF90CF90BF9067
:100EB000AF909F908F907F906F905F900895DC012E
:100EC0001296ED91FC911397E058FF4F819191910B
:100ED00080589F4F20813181821B930B60E870E026
:100EE0000E9472090895CF93DF93DC011296ED9171
:100EF000FC911397EF01CE57DF4F48815981E0589D
:100F0000FF4F80819181E058F0408417950719F4D4
:100F10002FEF3FEF0CC0E40FF51F2081CA010196AF
:100F200060E870E00E9472099983888330E0C9010B
:100F3000DF91CF910895FC01A085B18521898C9125
:100F400090E0022E02C0959587950A94E2F780FF03
:100F5000F6CF0484F585E02D6083089587E391E062
:100F6000909308028093070283E891E090930A022D
:100F70008093090285EC90E090930C0280930B0221
:100F800084EC90E090930E0280930D0280EC90E050
:100F90009093100280930F0281EC90E090931202E4
:100FA0008093110286EC90E09093140280931302D8
:100FB00084E08093150283E08093160287E080939B
:100FC000170285E08093180281E08093190208954A
:100FD0000F931F93CF93DF938C01EB0109C02196F0
:100FE000D801ED91FC910190F081E02DC8010995A7
:100FF00068816623A1F7DF91CF911F910F9108952A
:10100000EF92FF920F931F93CF93DF938C017B019D
:10101000EA010CC0D7016D917D01D801ED91FC91E1
:101020000190F081E02DC80109952197209791F753
:10103000DF91CF911F910F91FF90EF9008950F9343
:101040001F938C01DC01ED91FC910190F081E02D6A
:101050006DE00995D801ED91FC910190F081E02DB2
:10106000C8016AE009951F910F9108952F923F9250
:101070004F925F926F927F928F929F92AF92BF92A8
:10108000CF92DF92EF92FF920F931F93DF93CF9354
:10109000CDB7DEB7A0970FB6F894DEBF0FBECDBFB9
:1010A0001C016A017B01411551056105710549F477
:1010B000DC01ED91FC910190F081E02D60E3099558
:1010C00054C0882499245401422E55246624772440
:1010D00001E010E00C0F1D1F080D191DC701B6011E
:1010E000A30192010E948509F80160830894811C84
:1010F000911CA11CB11CC701B601A30192010E9461
:101100008509C901DA016C017D01C114D104E10432
:10111000F104F1F681E0E82EF12CEC0EFD1EE80C56
:10112000F91C3E010894611C711CD501C401019792
:10113000A109B1096C01C818D90814C0F601EE0D57
:10114000FF1D60816A3010F4605D01C0695CD101EF
:10115000ED91FC910190F081E02DC1010995089479
:10116000E108F1086E147F0449F7A0960FB6F894D1
:10117000DEBF0FBECDBFCF91DF911F910F91FF90CA
:10118000EF90DF90CF90BF90AF909F908F907F9027
:101190006F905F904F903F902F900895EF92FF9245
:1011A0000F931F93CF93DF93EC017A018B0177FFAD
:1011B0000FC0E881F9810190F081E02D6DE2099581
:1011C00010950095F094E094E11CF11C011D111D97
:1011D000CE01B801A7012AE00E943608DF91CF9125
:1011E0001F910F91FF90EF900895DC0121153105BB
:1011F00041F4ED91FC910190F081E02D642F09956F
:1012000008952A30310519F40E94CE0808950E94ED
:10121000360808952F923F924F925F926F927F927D
:101220008F929F92AF92BF92CF92DF92EF92FF92F6
:101230000F931F93DF93CF93CDB7DEB73B014C01E4
:1012400019012A016D897E898F89988D6A197B0918
:101250008C099D09621A730A840A950AA4019301F4
:101260000E945309E218F30804091509A80197011F
:101270000E94A7092A0D3B1D4C1D5D1DB901CA0125
:10128000CF91DF911F910F91FF90EF90DF90CF9062
:10129000BF90AF909F908F907F906F905F904F9096
:1012A0003F902F900895629FD001739FF001829F1D
:1012B000E00DF11D649FE00DF11D929FF00D839FE5
:1012C000F00D749FF00D659FF00D9927729FB00D82
:1012D000E11DF91F639FB00DE11DF91FBD01CF0195
:1012E0001124089597FB092E07260AD077FD04D014
:1012F00049D006D000201AF4709561957F4F08956B
:10130000F6F7909581959F4F0895A1E21A2EAA1B9A
:10131000BB1BFD010DC0AA1FBB1FEE1FFF1FA217A5
:10132000B307E407F50720F0A21BB30BE40BF50BA2
:10133000661F771F881F991F1A9469F7609570952B
:10134000809590959B01AC01BD01CF01089597FB5D
:10135000092E05260ED057FD04D0D7DF0AD0001C79
:1013600038F450954095309521953F4F4F4F5F4F42
:101370000895F6F790958095709561957F4F8F4F02
:101380009F4F0895AA1BBB1B51E107C0AA1FBB1F9B
:10139000A617B70710F0A61BB70B881F991F5A9501
:1013A000A9F780959095BC01CD010895EE0FFF1F20
:0C13B0000590F491E02D0994F894FFCF13
:1013BC0009007807EC07F609780700001000100008
:1013CC00100008002000F60E200005000100102778
:1013DC000000E8036400881300000D000300040003
:0E13EC00080001000000009B07E80700080051
:00000001FF
